:020000020000FC
:0E0000000C9425010C943700434C4B322E35E6
:040014000C94EC005C
:040034000C94B70071
:040040000C946F00AD
:040048000C94D60836
:100050000C94A7085A9A0E9446090E85002311F4B1
:1000600002E001C003E000936900E89A08950F934D
:100070000FB71F930F9394600F911F910FBF0F91B4
:10008000189507E005BBF4BC05E005BD089501E047
:1000900005BBA1E3B1E0AAA7BBA7A0E0B0E0A09395
:1000A0004D01B0934E0100E006BD01E000936E00EB
:1000B000089501E005BBA0E0B0E0AAA7BBA7AFEDA3
:1000C000B1E1A0934D01B0934E0100E006BD01E007
:1000D00000936E00089500E000936E0008950F9362
:1000E00078940FB70F93BF93AF93AAA5BBA50A2F20
:1000F0000B2B99F01197AAA7BBA779F4A0914D01FA
:10010000B0914E010A2F0B2B002309F4E4DF0CA55C
:10011000002319F498600FEF0AA3A0914D01B0914C
:100120004E010A2F0B2B002379F01197A0934D015C
:10013000B0934E0149F4E0924F01AAA5BBA50A2F46
:100140000B2B002309F4C7DFAF91BF910F910FBFB5
:100150000F91189504E0009381000AEF0093850049
:100160000AEE0093840001E000936F0008950F935E
:100170000AEE009384000AEF0093850078940FB78D
:100180001F930F930F810A9511F4906808850F83D0
:1001900009890A9511F490640FE0098B0DA500FF01
:1001A00008C00EA50A950EA721F40E7F0DA706D054
:1001B00022D00F911F910FBF0F91189510E8109347
:1001C0006D0014E010936800089510E010936D0026
:1001D00010E01093680008950F930FB71F930F93CB
:1001E000F4DF13E01EA71DA511601DA70F911F913D
:1001F0000FBF0F9118951F930F934F9B09C06BDF93
:100200000AA1002339F00F3F29F09260FAA202C040
:10021000EAA23DDF0F911F910895A89504B7077FCB
:1002200004BF00916000086100936000F0926000DC
:100230000895F894A895009160000861009360000B
:100240000AE00093600078940895589A599AE5DF7F
:10025000CEE1D1E0FF24EE24E3949927BB24CC2403
:10026000FDA6FEA6FCA6FB86FC8AFAA2FBA20FEF67
:100270000E8BFF8AF0924F01FDA2FEA2FA8AFB8A42
:10028000F9A6F8A6E6EBF3E1E0930001F093010193
:10029000FFA2E6E4F5E1E0930201F0930301EAE056
:1002A000FCE1E0931A01F0931B01E2EAF6E1E0932E
:1002B0000A01F0930B010CE308830EE30F83088718
:1002C0000FE0098B43D60E879AD634D60D8705E00A
:1002D000088FF98E32D60CA3002311F00FEF098F8F
:1002E00032D60F8736D609A301EC00936400C9DE2D
:1002F00031DFCED60E946D090ED7E0D2E8D25EDFA4
:1003000031D60F3F69F48827C5D48827CDD48827F4
:10031000D3D481E0D9D481E0DFD48827E5D4FCD5DB
:1003200006D60FA3002331F0E2EAF6E1E0930201E2
:10033000F093030105D60C87002311F40FE001C0F0
:1003400007E00A8709874FD4DBD1898031D067D491
:1003500009810815D9F30A95098360D17BDE789469
:10036000FFD2C8D4FDD2EDD623D090FD20D3FCCF50
:100370000F921F920F931F932F933F934F936F935F
:100380008F93BF93AF93FF93EF935F937F9310D0BF
:100390007F915F91EF91FF91AF91BF918F916F919D
:1003A0004F913F912F911F910F911F900F900895A2
:1003B000C5D091FF02C09D7F3CDF92FF11C00EA10E
:1003C000002311F42BD101C068D11CA510FF05C07A
:1003D00011FFFCD512FD01D601C0F8D59B7F098124
:1003E00097FF08C0E7D50EA1002311F417D101C073
:1003F00054D19F7796FF74C00A8900FF13C00B8900
:1004000000FD07C0E0EDF5E1E0930A01F0930B0178
:1004100006C0E2EAF6E1E0930A01F0930B010195D0
:1004200003950B8B0C890023A1F00D8900FD07C0FB
:10043000ECE3F6E1E0930C01F0930D0106C0E2EA73
:10044000F6E1E0930C01F0930D01019503950D8BFE
:1004500020C00E890E15E9F400914F01002331F000
:10046000FE8AFF8ACCD5F0924F0113C00F8900FDA0
:1004700007C0E2E2F6E1E0930C01F0930D0106C043
:10048000E2EAF6E1E0930C01F0930D01019503958A
:100490000F8B09A5002319F10B85002301F508A591
:1004A00000FD10C0E6EBF3E1E0930001F0930101E1
:1004B0000FA0002089F4E6E4F5E1E0930201F09357
:1004C00003010AC0E2EAF6E1E0930001F0930101C2
:1004D000E0930201F09303010195039508A79F7B28
:1004E00094FF24C0088D0A9511F477D505E0088F94
:1004F00009A1002311F001E036D30A89002341F05D
:10050000FA8AFB8AE2EAF6E1E0930A01F0930B0132
:100510009F7E95FF0BC019A10D8510230CA1102300
:1005200021F00B81043009F4EA8A9F7D93FF05C016
:10053000977F0E94D7070E94521408951127A0E0C8
:10054000B1E0A10FBF1DA10FBF1DED91FD9113954E
:100550000985039510170CF011C05D9A85918823C9
:10056000E1F3659145914423C1F34F3F41F3259158
:100570002F934F9305D08F916F91F4CF5D9A08958B
:10058000772794D55D9995D50FEFA82FA41B10F46C
:10059000AA95A027B62FB21B10F4BA95B0270A2F40
:1005A0000B1B50F47860862768278627422724276C
:1005B0004227AB27BA27AB277D7F042F081B08F4FF
:1005C00072607B7F022F061B08F4746055275D98CC
:1005D00073FD02C06ED501C085D58417C9F05B0FCD
:1005E00008F47F7E74FD0EC00A2F0894050B08F0F6
:1005F00009C07F7E5A1B08F4706172FD02C06395CA
:1006000001C06A9571FD02C08395E2CF8A95E0CF63
:1006100073FF03C086276827862708950F921F92CD
:100620001F930F933F932F93FF93EF934AD1088526
:100630000F831981139519831C3341F00BA10023FB
:1006400011F0FBA21EC083D0ECD01EC090611E85AD
:10065000112319F4EFD2C7D214C0F9821A8113956D
:100660001A831C334CF09062FA821B8113951B8312
:10067000183114F0FB8205C01DA1112311F4F7D22B
:10068000B2D243D070D0F8D0EF91FF912F913F912B
:100690000F911F911F900F9008951E85112329F12E
:1006A00010D108850F8319811A9519831F3F41F0D6
:1006B0000BA1002311F0FBA215C049D0B2D015C088
:1006C0001BE3198390611A811A951A831F3F51F415
:1006D0001BE31A8390621B811A951B831F3F11F441
:1006E00017E11B8312D03FD0C7D008951DA10EA1E2
:1006F000102B29F49FD209D036D0BED0089508958A
:1007000099D203D030D0B8D0089521D0E2EDF7E1EE
:100710000A8129E0029FE00DF11DE0930601F093AC
:100720000701EEEEF9E10A811CE07ED40F930B8104
:100730007BD4022F25E0029F1F91100D29E0129F0C
:10074000E00DF11DE0930801F09309010895E6EA38
:10075000F6E1098115E0019FE00DF11DE093040130
:10076000F093050108955DD00A811AE05DD4000F71
:100770000F84002019F0E6EBFEE102C0E0E6F2E2B1
:10078000E00FFF1D05911491000F111F009314013C
:1007900010931501022F000F0F84002019F0E8EDCF
:1007A000FDE102C0E2E8F1E2E00FFF1D05911491C6
:1007B000000F111F00931201109313010B810F847E
:1007C00000FC05C0EEEEF3E2E00FFF1D04911AE01D
:1007D0002BD4000F0F84002019F0E4E0F0E202C0F7
:1007E000EEEAF3E2E00FFF1D05911491000F111FD7
:1007F0000093180110931901022F000F0F8400209D
:1008000019F0E6E2FFE102C0E0EDF2E2E00FFF1DC9
:1008100005911491000F111F0093160110931701F9
:10082000089509811AE000D4000F0F84002019F008
:10083000E8E6FDE102C0E2E1F1E2E00FFF1D059113
:100840001491000F111F0093100110931101022F3A
:10085000000F0F84002019F0EAE8FCE102C0E4E395
:10086000F0E2E00FFF1D05911491000F111F00939E
:100870000E0110930F0108950F85002391F4E6E314
:10088000FCE1E0931A01F0931B01EEE6FCE10B8121
:100890000C3014F0EAE7FCE1E0931C01F0931D0139
:1008A0000CC0EAE0FCE1E0931A01F0931B01E2EADC
:1008B000F6E1E0931C01F0931D010895569A5E98AD
:1008C00008950D8500FF4E9A08955E9808955798F3
:1008D0005F9A08950F9309818EE1080F0C330CF095
:1008E0000C53CED4882329F443DD8981081729F0DD
:1008F000F8CF84D4C6D30F91089588E50F91089559
:100900008F93C2D4882311F433DDFBCF8F916DD444
:100910000895BAD4882311F42BDDFBCF8AD408952F
:100920008F93B2D4882311F423DDFBCF8F9118D09D
:100930000895AAD4882311F41BDDFBCF8AD408952F
:100940000F93A2D4882311F413DDFBCF0F91002362
:1009500019F0E6EEF5E26DC4EAEEF5E26AC4089538
:10096000E2EEF5E266C412E0BDD48F7768D38395DA
:1009700083958C330CF08C53082E00E4F9DC0A9537
:100980000023E1F712E0AED48F7759D30816A9F708
:100990000895E9DFE8DF0895FCDFFBDF0895B9DFA4
:1009A000BFDFE1DF0895B5DFBBDFF3DF08958F938D
:1009B0001F930F933F932F93BF93AF93FF93EF93A7
:1009C0000F921F921BD45DD3883509F08BC0ECE3E6
:1009D000F4E29FDF7FDF94DFA3DF8435C9F1843445
:1009E00009F468C0833509F463C08C3411F427D24C
:1009F00079C0813411F4F3D175C0863511F456D223
:100A000071C0833411F491D16DC08E3411F404D2CD
:100A100069C0803511F423D265C0823411F42DD21F
:100A200061C0813511F4B2D15DC0823511F4C6D1F7
:100A300059C0863411F444D255C0873511F4ACDF67
:100A400051C0883411F4ECD24DC0883569F1BFCF64
:100A5000E6E6F4E25EDF54D030F12ED161DFEEE75E
:100A6000F4E257DF4DD0F8F01FD15ADFE6E9F4E2A7
:100A700050DF46D0C0F00E85002351F48F9389815A
:100A80008F935CDD8F91CBD009810817C9F38F91CB
:100A900001D1EBA209810A950983C0DD9B7740DF74
:100AA000002761D004C02CDEE8EBF5E232DF1AC08B
:100AB00021D118C0EEEAF4E22CDF22D0A8F314D141
:100AC0002FDFE6ECF4E225DF1BD070F305D128DF41
:100AD000EEEDF4E21EDF14D038F3F6D021DF00276C
:100AE00042D000C01DDFEBA21F900F90AF91BF91CD
:100AF000EF91FF912F913F910F911F918F91089549
:100B0000E9DEFEDE883511F4089408950DD0C0F3B7
:100B1000082FE0DEF5DE8835B9F306D0D0F31AE011
:100B2000019F800D88940895803328F08A3318F44B
:100B300080538894089508940895E6E1F4E2E9DE8C
:100B400082E3DEDE8EE2DCDE85E3DADEE9DE0895D6
:100B500086D28F9382958F708AD28D938F918F706A
:100B600086D28D93089590D3882311F401DCFBCFB6
:100B7000FF93EF93BF93AF930F93A0E5B1E08C8108
:100B8000E7DF8DE28D938D81EEEEF5E28A95880F99
:100B9000880FE80FFF1D85918D9385918D93859129
:100BA0008D938DE28D9382E38D9380E38D938E817F
:100BB000CFDF80E28D938B81CBDF8AE38D938A81B7
:100BC000C7DF8AE38D938981C3DF0F91002321F072
:100BD0008DE08D938AE08D93FD923BD3AF91BF91D1
:100BE000EF91FF9108950F938F9315E07BD38F734F
:100BF00026D280320CF08E2D8C8317E073D38F7148
:100C00001ED28D300CF08E2D8D8318E06BD317D251
:100C100083360CF088278E838F910F9108958F93E0
:100C200012E060D38F770BD28C330CF08827898346
:100C30008F9108958F9312E055D387FDA2D18F77BE
:100C4000FED18C330CF08827898313E04BD38F7748
:100C5000F6D18C330CF088278A8314E043D38F734A
:100C6000EED188310CF088278B838F9108958CA565
:100C7000882379F48981F3D112E0082F4CD38A813B
:100C8000EED113E0082F47D38B81E9D114E0082F70
:100C900042D308958F93082F0C3320F48983DFD13A
:100CA00012E039D38F910895082F0C3320F48A83F2
:100CB000D6D113E030D30895082F083120F48B8368
:100CC000CED114E028D30895082F003220F48C836D
:100CD000C6D115E020D30895082F0C3020F48D8361
:100CE000BED117E018D30895082F8E83B8D118E02D
:100CF00012D3089522DF002736DF80E201DE82E58D
:100D00000E85002309F081E4FBDD0D85002311F43D
:100D10008CE4F6DD0CA1002311F482E4F1DD09A1DD
:100D2000002311F086E5ECDD08952F93E6EFF4E261
:100D3000F0DD0B85002339F0C3D2002722271A8566
:100D4000E6EBF3E109C015D0B7D20E2D2FEFBB248F
:100D5000CC2411E0E8E8F6E11987E0930001F09374
:100D600001011CA1112309F4298F0B87E9DD2F91C3
:100D700008950DA1002321F01EE318871F83FDA213
:100D80000EA1002309F0FEA2B1DC08950E8500FD3E
:100D900004C0E6E7F5E2BDDD10C0ECE5F5E2B9DD43
:100DA0000DA1002319F01EE3002702C012E00E2D52
:100DB00018871F830DA3C4DD99DC08950E8500FDFF
:100DC00004C0E6E7F5E2A5DD09C0E8E6F5E2A1DD4D
:100DD0000EA1019503950EA3B3DD88DC0895E6E32B
:100DE000F5E297DD0E85002349F0C3DF0027E2EA34
:100DF000F6E1E0930C01F0930D0107C00395E6E1E5
:100E0000F6E1E0930C01F0930D010E877CD098DDA4
:100E10000CA500FF0EDA0895ECE0F5E27ADD0C8512
:100E2000002319F000271FE002C0039517E00C878C
:100E300019871A8765D00195039582DD0895EEE143
:100E4000F5E267DD0D85002311F0002702C0039550
:100E50003CDD0D874FD00195039572DD0895EEE2DC
:100E6000F5E257DD0F85019503950F874FD001956A
:100E7000039566DD01DD77DC0895E8E4F5E249DD00
:100E80000CA1019503950CA30F9337D00195039501
:100E900057DD0F911B85112341F4002329F00FEF3B
:100EA000098FBB24CC2401C0F98E0895E4E2F5E259
:100EB00030DD09A10195039509A32BD041DD0895EB
:100EC000E4EAF5E226DD0FA1002321F00027E6E4A5
:100ED000F5E103C00395E2EAF6E1E0930201F09345
:100EE00003010FA304D0019503952ADD0895A7E01F
:100EF000B0E016C0A0E0B0E013C0A6E0B0E010C0C3
:100F0000A3E0B0E00DC0A2E0B0E00AC0A4E0B0E011
:100F100007C0A1E0B0E004C0A5E0B0E001E000C07F
:100F20000CA4002019F400BD16E021D00895A7E01C
:100F3000B0E012C0A0E0B0E00FC0A6E0B0E00CC08E
:100F4000A3E0B0E009C0A4E0B0E006C0A2E0B0E0D9
:100F500003C0A1E0B0E000C011E009D00F3F09F4E8
:100F600000270895A5E0B0E011E001D00895A1BDEB
:100F7000B2BD119611FDFA9A1FBBF999FECF00B5CB
:100F800008950E890F3F49F4EE8AEF8AE2E2F6E116
:100F9000E0930C01F0930D018CD80895EE8AEF8A4E
:100FA000E2E2F6E1E0930C01F0930D010895FE8A70
:100FB000FF8A25D00DA100FD0895EC8AED8AECE3AF
:100FC000F6E1E0930C01F0930D0108950C8900FF08
:100FD0000895FC8AFD8A13D00895098D0F3F71F0A2
:100FE000FF93EF93E6E0F4E203950770098F000F9B
:100FF000E00FFF1DB590C490EF91FF9108950E850D
:10100000002339F4E2EAF6E1E0930C01F0930D01DC
:1010100006C0E6E1F6E1E0930C01F0930D010895BE
:10102000EEE1F6E276DC0895222738E0000F221F79
:10103000211710F00395211B3A95C1F708950F92DF
:101040001F920F938F9382958F700AE0809F002DDF
:101050008F918F70800F0F911F900F900895082F20
:101060001AE0E2DF07700295022B802F0895FF93AC
:10107000EF93EEEDF3E2E80FFF1D8491EF91FF9106
:101080000895813624F08B3710F400E2801B089518
:10109000209A219A229A239A389A399A3A9A3B9A14
:1010A000539A549A559A5D9A5C9A089538B1307F54
:1010B00008958F938B0D5B98082F8F70832B88B9C1
:1010C000029505B9862F81958C0D082F8F70832B83
:1010D00002955C985C9A5B9A88B905B95C985C9AB1
:1010E0008F9108956F936B0D5B98062F6F70632B34
:1010F00068B9029505B9682F61956C0D062F6F7060
:10110000632B02955C985C9A5B9A68B905B95C9808
:101110005C9A6F91089510E41093C400F092C5009A
:10112000F092C00018E41093C10016E01093C200C2
:10113000F8A2EA8EFE8EFF8EFB8EFC8E1FEF1D8FB7
:1011400008951091C10010691093C1000895AFB6C1
:101150000F931F93FF93EF930D8D0F3F79F003953E
:10116000E0E5F1E0E00FFF1D1081112319F40FEF0E
:10117000EA8E02C01093C6000D8F12C0EB8DFC8D5D
:101180000E2F0F2B39F0EF5FFF4F1491112321F435
:10119000FB8EFC8EEA8E04C01093C600EB8FFC8F92
:1011A000EF91FF911F910F91AFBE1895AFB60F93BE
:1011B0001F932F933F93FF93EF932091C6000E8DC3
:1011C000302F03950F701F8D011739F00E8FE0ED52
:1011D000F1E0E30FFF1D20839160EF91FF913F91BC
:1011E0002F911F910F91AFBE18950F930A8D002379
:1011F000E9F3FA8E8093C6000F91089590FFFECF19
:101200000F931F93FF93EF931E8D0F8D8827011768
:1012100051F0E0EDF1E0E00FFF1D808103950F70CC
:101220000F8F011709F49E7FEF91FF911F910F918E
:1012300008950F93FF93EF930A8D0023E9F3FA8E3D
:10124000EB8FFC8F04910093C600EF91FF910F91FB
:1012500008950F93FF93EF930A8D0023E9F3FA8E1D
:10126000FD8EE0E5F1E00081002321F40FEF0D8F0A
:10127000EA8E02C00093C600EF91FF910F9108958E
:10128000882790FD839508958A8D08951F930F9365
:1012900017D01FE000E43FD01EE001E83CD011E091
:1012A00001E139D00F911F9108951FE000E433D080
:1012B00011E001E130D008951DE000E82CD0089540
:1012C0001DE0002728D00895000000000000000065
:1012D000000000000000000008953C9A3D9A449AE6
:1012E000459A08955ED0F0DF02EA36D0EDDF2AD0CD
:1012F000C8F3012F31D0E8DF25D0A0F34CD051D076
:1013000003EA2AD0E1DF1ED068F333D0449A459A2D
:1013100042D0802F089545D0D7DF0F9302EA1CD02A
:10132000D3DF10D00F91B8F30F93012F15D00AD04F
:101330000F9188F30F9310D005D00F9160F3000048
:101340002AD008953C98449A0894459ABDDF349B6E
:10135000889445983C9A08953F9338E0449A000F4A
:1013600008F04498459AB0DF45983A95B9F73F910F
:1013700008953F933C98449A00E038E0459A0894D9
:10138000A3DF349B8894001F45989EDF3A95B1F700
:101390003C9A3F9108954498459A00000000449A71
:1013A0000895449A459A0000000044980000000007
:1013B0004598000008957A157A27008018831589CA
:1013C000158C188C1B80278C270086DC83D97DD94F
:1013D0007ADC7AE87DEB83EB86E886E583E27DE2E2
:1013E0007AE500E07AE377E977EC7AEC7DE980EC66
:1013F00083EC86E989E389E08600E380E980001FC9
:101400007D1C801C801680137D137A16771C771F35
:101410007A1F861C8916891386008002800E008D33
:10142000028C07009A04990900A608A50C00B30CC9
:10143000B11100BF12BA1B00CA1AC71E00D422D0B5
:101440002600DD2BD92F00E535E13800ED41E446DB
:1014500000F34CEE4E00F759F35A00FB65F66600B8
:10146000FD72F87300FD80F18000FD8DF88C00FBAB
:101470009AF69900F7A6F3A500F3B3EEB100EDBF1D
:10148000E4BA00E5CAE1C700DDD4D9D000D4DDD08C
:10149000D900CAE5C7E100BFEDBAE400B3F3B1EE8D
:1014A00000A6F7A5F3009AFB99F6008DFD8CF800D5
:1014B0007FFD7FF10072FD73F80065FB66F6005951
:1014C000F75AF3004CF34EEE0041ED46E40035E5EB
:1014D00038E1002BDD2FD90022D426D0001ACA1EF5
:1014E000C70012BE1BB9000CB311B10008A60CA5B1
:1014F00000049A099900028D078C00027F0E7F007C
:101500000272077300046509660008590C5A000C42
:101510004C114E0012411B46001A351E3800222B7A
:10152000262F002B222F2600351A381E0040124588
:101530001B004C0C4E110059085A0C00650466093A
:101540000072027307FFB51CB52E0000D245D542CC
:10155000DB42DE45DE48D254DE540000E0B4D4B4B1
:10156000DDABDDBD0000B8CFACCFACD8B5D8B8DBB3
:10157000B8DEB5E1AFE1ACDE000047CF53CF53D2C8
:1015800050D54DDB4DE1000022B41FB11FAE22ABA0
:1015900028AB2BAE2BB128B422B41FB71FBA22BD83
:1015A00028BD2BBA2BB728B40000214221540000DB
:1015B00027452A4230423345335130542A5427516B
:1015C00027450000491C492E0000531C532EFF00E4
:1015D000B25CB25ABA5ABA66B266B26400BE66BEAD
:1015E00062C462C466BE6600C466C45A00C966C9E5
:1015F0005ACD5ACF5CCF60CD62C96200CD62CF6652
:10160000FF007E467E3A823A843C844082427E429B
:101610000082428446FF7C46803A84460082427EB5
:1016200042FF7C467C3A823A843C843E82407C4045
:1016300082408442844482467C46FF007E467E3A55
:10164000823A843C843E82407E40FF00A764AD64C1
:10165000AF66AF6EAD70A770A76400BB64B364B330
:1016600070BB7000B96AB36A00BE70BE64C268C65F
:1016700064C67000C966CB64CF64D166D16ECF708A
:10168000CB70C96EC966FF0001FE0101FE01FEFEBE
:1016900001FEFE010101FEFE01FE0101FE01FEFE52
:1016A000FF000101FF0080148080FF8B148080FF09
:1016B00096168080FFA1198080FFAB1D8080FFB649
:1016C000228080FFBF288080FFC82F8080FFD03716
:1016D0008080FFD7408080FFDD4A8080FFE2548019
:1016E00080FFE65E8080FFE9698080FFEB74808088
:1016F000FFEB808080FFEB8B8080FFE9968080FF8E
:10170000E6A18080FFE2AB8080FFDDB68080FFD75E
:10171000BF8080FFD0C88080FFC8D08080FFBFD747
:101720008080FFB6DD8080FFABE28080FFA1E68095
:1017300080FF96E98080FF8BEB8080FF7FEB8080CD
:10174000FF74EB8080FF69E98080FF5EE68080FFA8
:1017500054E28080FF4ADD8080FF40D78080FF37E1
:10176000D08080FF2FC88080FF28BF8080FF22B5F7
:101770008080FF1DAB8080FF19A18080FF169680BE
:1017800080FF148B8080FF147F8080FF1474808022
:10179000FF16698080FF195E8080FF1D548080FFE6
:1017A000224A8080FF28408080FF2F378080FF37CB
:1017B0002F8080FF40288080FF49228080FF541DB9
:1017C0008080FF5E198080FF69168080FF7414801E
:1017D00080FF8280801A7E808280FF81808A1A7ECC
:1017E0007F8180FF8180951C7E7F8180FF81809F2B
:1017F0001E7E7F8180FF8180A9227E7F8180FF8184
:1018000081B3277E7E8181FF8181BB2D7E7E818198
:10181000FF8181C4347E7E8181FF8181CB3B7E7ECE
:101820008181FF8181D2447E7E8181FF8081D84D7C
:101830007F7E8081FF8081DD567F7E8081FF808179
:10184000E1607F7E8081FF8081E36A7F7E8081FF0F
:101850008081E5757F7E8081FF7F82E580807E7F4D
:1018600082FF7F81E58A807E7F81FF7F81E3958093
:101870007E7F81FF7F81E19F807E7F81FF7F81DD91
:10188000A9807E7F81FF7E81D8B3817E7E81FF7EAD
:1018900081D2BB817E7E81FF7E81CBC4817E7E81B1
:1018A000FF7E81C4CB817E7E81FF7E81BBD2817E23
:1018B0007E81FF7E81B3D8817E7E81FF7E80A9DD1F
:1018C000817F7E80FF7E809FE1817F7E80FF7E80A2
:1018D00095E3817F7E80FF7E808AE5817F7E80FF29
:1018E0007E7F7FE582807E7FFF7E7F75E581807EC3
:1018F0007FFF7E7F6AE381807E7FFF7E7F60E18164
:10190000807E7FFF7E7F56DD81807E7FFF7E7F4DE4
:10191000D881807E7FFF7E7E44D281817E7EFF7E65
:101920007E3BCB81817E7EFF7E7E34C481817E7E44
:10193000FF7E7E2DBB81817E7EFF7F7E27B28081F0
:101940007F7EFF7F7E22A980817F7EFF7F7E1E9F1C
:1019500080817F7EFF7F7E1C9580817F7EFF7F7EE2
:101960001A8A80817F7EFF807E1A7F7F82807EFF41
:10197000807E1A757F81807EFF807E1C6A7F8180D9
:101980007EFF807E1E607F81807EFF807E22567F6C
:1019900081807EFF807E274D7F81807EFF817E2D2E
:1019A000447E81817EFF817E343B7E81817EFF810A
:1019B0007E3B347E81817EFF817E442D7E81817ECF
:1019C000FF817E4C277E81817EFF817F56227E8033
:1019D000817FFF817F601E7E80817FFF817F6A1C07
:1019E0007E80817FFF817F751A7E80817FFF82806C
:1019F00080447E808280FF818086447E7F8180FF5C
:101A000081808C457E7F8180FF818092467E7F81B0
:101A100080FF818098497E7F8180FF81819E4C7EFE
:101A20007E8181FF8181A34F7E7E8181FF8181A89C
:101A3000537E7E8181FF8181AC577E7E8181FF81D3
:101A400081B05C7E7E8181FF8081B3627F7E8081F8
:101A5000FF8081B6677F7E8081FF8081B96D7F7E48
:101A60008081FF8081BA737F7E8081FF8081BB7916
:101A70007F7E8081FF7F82BB80807E7F82FF7F812F
:101A8000BB86807E7F81FF7F81BA8C807E7F81FFD5
:101A90007F81B992807E7F81FF7F81B698807E7F33
:101AA00081FF7E81B39E817E7E81FF7E81B0A38196
:101AB0007E7E81FF7E81ACA8817E7E81FF7E81A8B3
:101AC000AC817E7E81FF7E81A3B0817E7E81FF7EA0
:101AD000819EB3817E7E81FF7E8098B6817F7E80ED
:101AE000FF7E8092B9817F7E80FF7E808CBA817F6D
:101AF0007E80FF7E8086BB817F7E80FF7E7F7FBB76
:101B000082807E7FFF7E7F79BB81807E7FFF7E7FAC
:101B100073BA81807E7FFF7E7F6DB981807E7FFF7B
:101B20007E7F67B681807E7FFF7E7F62B381807E0D
:101B30007FFF7E7E5CB081817E7EFF7E7E57AC81A2
:101B4000817E7EFF7E7E53A881817E7EFF7E7E4FDA
:101B5000A381817E7EFF7F7E4C9D80817F7EFF7F83
:101B60007E499880817F7EFF7F7E469280817F7E46
:101B7000FF7F7E458C80817F7EFF7F7E44868081D3
:101B80007F7EFF807E447F7F82807EFF807E4479DF
:101B90007F81807EFF807E45737F81807EFF807E97
:101BA000466D7F81807EFF807E49677F81807EFFDA
:101BB000807E4C627F81807EFF817E4F5C7E818152
:101BC0007EFF817E53577E81817EFF817E57537ECB
:101BD00081817EFF817E5C4F7E81817EFF817E617F
:101BE0004C7E81817EFF817F67497E80817FFF817E
:101BF0007F6D467E80817FFF817F73457E80817F00
:101C0000FF817F79447E80817FFF6EAD6EAB70ABCC
:101C100070AD6EAD006EB16EB370B370B16EB100E9
:101C20008FAD8FAB91AB91AD8FAD008FB18FB39175
:101C3000B391B18FB1FF62AD62AB64AB64AD62AD25
:101C40000062B162B364B364B162B10082AD82ABD1
:101C500084AB84AD82AD0082B182B384B384B1829F
:101C6000B100AEB5AEA9B2ADB6A9B6B5FF00A2B58A
:101C7000A6A9AAB500A8B1A4B1FFA4B5A4A9A8A912
:101C8000AAABAAADA8AFA4AFFF004F0E590E5C0ED1
:101C9000640E720E770E810E8E0E950EA60EA2ABFE
:101CA000A4A9A8A9AAABAAB3A8B5A4B5A2B3A2AB8C
:101CB000FF00A6A9A6B5FF00A2ABA4A9A8A9AAAB3C
:101CC000AAADA2B5AAB5FF00A2ABA4A9A8A9AAABC8
:101CD000AAADA8AFAAB1AAB3A8B5A4B5A2B300A4EF
:101CE000AFA8AFFFAAAFA2AFA8A9A8B5FF00AAA945
:101CF000A2A9A2AFA8AFAAB1AAB3A8B5A4B5A2B32E
:101D0000FF00AAABA8A9A4A9A2ABA2B3A4B5A8B589
:101D1000AAB3AAB1A8AFA4AFA2B1FF00A2A9AAA971
:101D2000AAABA8ADA6B1A6B5FF00A4AFA2ADA2AB69
:101D3000A4A9A8A9AAABAAADA8AFA4AFA2B1A2B307
:101D4000A4B5A8B5AAB3AAB1A8AFFF00AAADA8AF21
:101D5000A8AFA4AFA2ADA2ABA4A9A8A9AAABAAB3ED
:101D6000A8B5A4B5A2B3FF00BA0EC40EC70ECF0E1D
:101D7000DD0EE20E96AB98A99CA99EAB9EB39CB5D6
:101D800098B596B396ABFF009AA99AB5FF0096ABAB
:101D900098A99CA99EAB9EAD96B59EB5FF0096AB4B
:101DA00098A99CA99EAB9EAD9CAF9EB19EB39CB5DD
:101DB00098B596B30098AF9CAFFF9EAF96AF9CA925
:101DC0009CB5FF009EA996A996AF9CAF9EB19EB30D
:101DD0009CB598B596B3FF00F60E000F030F0B0FDE
:101DE000190F1E0F280F350F3C0F4D0F82AB84A922
:101DF00088A98AAB8AB388B584B582B382ABFF0069
:101E000086A986B5FF0082AB84A988A98AAB8AAD72
:101E100082B58AB5FF0082AB84A988A98AAB8AAD56
:101E200088AF8AB18AB388B584B582B30084AF889D
:101E3000AFFF8AAF82AF88A988B5FF008AA982A9BF
:101E400082AF88AF8AB18AB388B584B582B3FF0008
:101E50008AAB88A984A982AB82B384B588B58AB3DA
:101E60008AB188AF84AF82B1FF0082A98AA98AAB08
:101E700088AD86B186B5FF0084AF82AD82AB84A900
:101E800088A98AAB8AAD88AF84AF82B182B384B5AA
:101E900088B58AB38AB188AFFF008AAD88AF88AFB2
:101EA00084AF82AD82AB84A988A98AAB8AB388B596
:101EB00084B582B3FF00610F6B0F6E0F760F840F36
:101EC000890F76AB78A97CA97EAB7EB37CB578B55B
:101ED00076B376ABFF007AA97AB5FF0076AB78A926
:101EE0007CA97EAB7EAD76B57EB5FF0076AB78A9DA
:101EF0007CA97EAB7EAD7CAF7EB17EB37CB578B580
:101F000076B30078AF7CAFFF7EAF76AF7CA97CB5AF
:101F1000FF007EA976A976AF7CAF7EB17EB37CB59B
:101F200078B576B3FF009D0FA70FAA0FB20FC00FB1
:101F3000C50FCF0FDC0FE30FF40F62AB64A968A9E4
:101F40006AAB6AB368B564B562B362ABFF0066A9F9
:101F500066B5FF0062AB64A968A96AAB6AAD62B5F9
:101F60006AB5FF0062AB64A968A96AAB6AAD68AFE5
:101F70006AB16AB368B564B562B30064AF68AFFFB5
:101F80006AAF62AF68A968B5FF006AA962A962AFCB
:101F900068AF6AB16AB368B564B562B3FF006AAB93
:101FA00068A964A962AB62B364B568B56AB36AB183
:101FB00068AF64AF62B1FF0062A96AA96AAB68AD9D
:101FC00066B166B5FF0064AF62AD62AB64A968A993
:101FD0006AAB6AAD68AF64AF62B162B364B568B54D
:101FE0006AB36AB168AFFF006AAD68AF68AF64AF4B
:101FF00062AD62AB64A968A96AAB6AB368B564B53F
:1020000062B3FF0005100F10121055AB57A95BA962
:102010005DAB5DB35BB557B555B355ABFF0059A983
:1020200059B5FF0055AB57A95BA95DAB5DAD55B583
:102030005DB5FF0024102E103110391047104C10E0
:10204000561063106A107B1096AB98A99CA99EABA2
:102050009EB39CB598B596B396ABFF009AA99AB576
:10206000FF0096AB98A99CA99EAB9EAD96B59EB578
:10207000FF0096AB98A99CA99EAB9EAD9CAF9EB16C
:102080009EB39CB598B596B30098AF9CAFFF9EAF3A
:1020900096AF9CA99CB5FF009EA996A996AF9CAF50
:1020A0009EB19EB39CB598B596B3FF009EAB9CA91C
:1020B00098A996AB96B398B59CB59EB39EB19CAFCC
:1020C00098AF96B1FF0096A99EA99EAB9CAD9AB120
:1020D0009AB5FF0098AF96AD96AB98A99CA99EAB18
:1020E0009EAD9CAF98AF96B196B398B59CB59EB394
:1020F0009EB19CAFFF009EAD9CAF9CAF98AF96ADDC
:1021000096AB98A99CA99EAB9EB39CB598B596B387
:10211000FF008F1099109C10A410B210B7108AAB5A
:102120008CA990A992AB92B390B58CB58AB38AABC7
:10213000FF008EA98EB5FF008AAB8CA990A992AB47
:1021400092AD8AB592B5FF008AAB8CA990A992ABEB
:1021500092AD90AF92B192B390B58CB58AB3008C2A
:10216000AF90AFFF92AF8AAF90A990B5FF0092A950
:102170008AA98AAF90AF92B192B390B58CB58AB369
:10218000FF00CB10D510D810E010EE10F310FD10AA
:102190000A111111221176AB78A97CA97EAB7EB30E
:1021A0007CB578B576B376ABFF007AA97AB5FF0037
:1021B00076AB78A97CA97EAB7EAD76B57EB5FF0007
:1021C00076AB78A97CA97EAB7EAD7CAF7EB17EB3C9
:1021D0007CB578B576B30078AF7CAFFF7EAF76AFD5
:1021E0007CA97CB5FF007EA976A976AF7CAF7EB1D5
:1021F0007EB37CB578B576B3FF007EAB7CA978A9B9
:1022000076AB76B378B57CB57EB37EB17CAF78AF74
:1022100076B1FF0076A97EA97EAB7CAD7AB17AB5A6
:10222000FF0078AF76AD76AB78A97CA97EAB7EADAA
:102230007CAF78AF76B176B378B57CB57EB37EB13E
:102240007CAFFF007EAD7CAF7CAF78AF76AD76AB78
:1022500078A97CA97EAB7EB37CB578B576B3FF0058
:102260003611401143114B1159115E116AAB6CA923
:1022700070A972AB72B370B56CB56AB36AABFF008C
:102280006EA96EB5FF006AAB6CA970A972AB72AD96
:102290006AB572B5FF006AAB6CA970A972AB72AD7A
:1022A00070AF72B172B370B56CB56AB3006CAF70D9
:1022B000AFFF72AF6AAF70A970B5FF0072A96AA9CB
:1022C0006AAF70AF72B172B370B56CB56AB3FF002C
:1022D00072117C117F11871195119A11A411B111FE
:1022E000B811C91156AB58A95CA95EAB5EB35CB519
:1022F00058B556B356ABFF005AA95AB5FF0056ABB6
:1023000058A95CA95EAB5EAD56B55EB5FF0056AB95
:1023100058A95CA95EAB5EAD5CAF5EB15EB35CB567
:1023200058B556B30058AF5CAFFF5EAF56AF5CA96F
:102330005CB5FF005EA956A956AF5CAF5EB15EB357
:102340005CB558B556B3FF005EAB5CA958A956AB57
:1023500056B358B55CB55EB35EB15CAF58AF56B11D
:10236000FF0056A95EA95EAB5CAD5AB15AB5FF003D
:1023700058AF56AD56AB58A95CA95EAB5EAD5CAF2D
:1023800058AF56B156B358B55CB55EB35EB15CAFED
:10239000FF005EAD5CAF5CAF58AF56AD56AB58A911
:1023A0005CA95EAB5EB35CB558B556B3FF00DA11FD
:1023B000E411E71149AB4BA94FA951AB51B34FB54C
:1023C0004BB549B349ABFF004DA94DB5FF0049AB33
:1023D0004BA94FA951AB51AD49B551B5FF003031B3
:1023E00032333435363738394142434445460C019F
:1023F00002030405060708090A0B0C010203040581
:10240000060708090A0B0000010001010001FF0195
:10241000FF00FFFF00FF447574636874726F6E699C
:102420007820415652204F7363696C6C6F73636FF1
:10243000706520436C6F636B20560000456E7465B9
:102440007220636F6D6D616E642028412C422C43B5
:102450002C442C462C482C4C2C4E2C502C532C54B9
:102460002C56293A0000456E74657220322064694A
:1024700067697420686F7572733A20202000456E7A
:102480007465722032206469676974206D696E75A5
:102490007465733A2000456E746572203220646959
:1024A000676974207365636F6E64733A2000456ECC
:1024B000746572203220646967697420796561727D
:1024C0003A2020202000456E746572203220646915
:1024D000676974206D6F6E74683A20202000456E25
:1024E0007465722032206469676974206461793A86
:1024F00020202020200043616C6962726174696F42
:102500006E205061747465726E2000004E756D65AA
:1025100072696320646973706C61792000004C45B6
:1025200044200000566572626F7365200000414DC3
:102530002F504D20000041565220436C6F636B209A
:102540004D617374657220004275726E2D696E2044
:1025500050726576656E74696F6E200046617374A3
:10256000204D6F64652000005265766572736520AA
:102570004D6F6465200052657175657374656420E4
:102580006D6F64652072657175697265732041565F
:102590005220636C6F636B204D6173746572204DC4
:1025A0006F646500416C6C204469676974732064D2
:1025B0006973706C6179200043616E63656C206F94
:1025C000722054696D656F7574004E6F7420456E8E
:1025D000746572696E672044656D6F204D6F646528
:1025E00000000D0A00004F6E00004F6666004A6151
:1025F0006E1F4665621C4D61721F4170721E4D61F7
:10260000791F4A756E1E4A756C1F4175671F5365A9
:10261000701E4F63741F4E6F761E4465631F4475B2
:1026200074636874726F6E6978204F7363696C6C41
:102630006F73636F706520436C6F636B2048656CCC
:10264000703A0D0A413A20546F67676C65204D61FE
:102650007374657220436C6F636B20626574776579
:10266000656E2041565220616E64205254430D0A1B
:10267000423A20546F67676C65204275726E2D690F
:102680006E2070726576656E74696F6E0D0A433ADE
:1026900020446973706C61792043616C6962726176
:1026A00074696F6E207061747465726E0D0A443ABD
:1026B000204368616E676520446174650D0A463A7F
:1026C00020546F67676C6520416C6C2044696769B2
:1026D000747320446973706C61790D0A4C3A20540C
:1026E0006F67676C65204C454420626C696E6B694E
:1026F0006E670D0A4E3A20546F67676C65204E7501
:102700006D6572696320446973706C6179200D0A8C
:10271000503A20546F67676C6520414D2F504D2013
:102720000D0A533A20446973706C617920537461C7
:10273000747573200D0A543A204368616E676520F2
:1027400054696D650D0A563A20546F67676C6520B1
:10275000566572626F7365204F75747075740D0ADB
:102760000000ECE4F6E1E0930A01F0930B01089518
:10277000E2EAF6E1E0930A01F0930B0108950C857B
:102780000023D9F50E940C0736C00C850023A9F15F
:102790000E940C0730C00F85002379F50E942F0797
:1027A0002AC00F85002349F10E942F0724C00FA1E2
:1027B000002319F50E9460071EC00FA10023E9F055
:1027C0000E94600718C00D850023B9F40E941F07FE
:1027D00012C00D85002389F00E941F070CC00B85D5
:1027E000002361F00E94950606C00B85002331F49A
:1027F0000E94950600C00E94900400C0089509A19F
:102800000023E1F30E945607F6CF09A10023B1F798
:102810000E945607F0CF0E85002381F30E94EF0639
:10282000EACF0E85002351F70E94EF06E4CF0DA1F9
:10283000002321F30E94C606DECF0DA10023F1F68E
:102840000E94C606D8CF0EA10023C1F20E94DE0668
:10285000D2CF0EA1002391F60E94DE06CCCF09A5AF
:102860000195039509A7E6EBF3E1E0930001F093EE
:1028700001010FA000FC0895E6E4F5E1E0930201F8
:10288000F093030108950895F98E08950E94E607D4
:1028900008950E94DA0708950E94D70708950E94BC
:1028A000CE07089501E00CA70E94B113C0DFCBDF73
:1028B00096DFE6E3FAE20E94CF04E6EBFAE20E943A
:1028C000CF040E94BF130E94D713E4EEFAE20E94E5
:1028D000CF040E94DD13E6E0FBE20E94CF040E94D9
:1028E000CB130E94C513E4E2FBE20E94CF040E94D6
:1028F000D113E6E4FBE20E94CF04E8E6FBE20E948B
:10290000CF040E94CB130E94B3040E94D7130E94ED
:10291000B3040E94D1130E94B3040E94DD130E94ED
:10292000BF130E94B3040E94DD130E94C5130E94CE
:10293000B3040E94D7130E94BF130E94B3040E94E5
:10294000DD130E94D1130E94C5130E94B3040E949C
:10295000E313E4E8FBE20E94D3040E94E913EEE9EA
:10296000FBE20E94D3040E94F513E2EBFBE20E941B
:10297000D3040E94EF13ECECFBE20E94D3040E940C
:102980001114EEEDFBE20E94D3040E941D14E0E15D
:10299000FCE20E94D3040E94C9040E941714E2E2E0
:1029A000FCE20E94D3040E942914E6E3FCE20E94A8
:1029B000D3040E941D14E8E4FCE20E94D3040E94A8
:1029C000C9040E94B90609E00CA70E944F14E6E86A
:1029D000FCE20E94D3040E94C90403E00CA70E94F9
:1029E0004C140E944914E8EDFCE20E94D3040E94BA
:1029F000C90401E10CA70E9446140E942F14E8E2CA
:102A0000FDE20E94D30405E00CA70E942F140E944F
:102A10004414E6E4FDE20E94D3040E94C904FCA62B
:102A20000E944314E6EAFDE20E94CF040E94B8131C
:102A30000E9419010895546869732064656D6F20C0
:102A40006D6F64652073686F777320736F6D652099
:102A50006F6620746865206361706162696C697477
:102A6000696573206F6620746865204475746368B7
:102A700074726F6E69780D0A415652204F73636904
:102A80006C6C6F73636F706520436C6F636B2E208B
:102A90004974207072657365727665732074686519
:102AA000207374617465206F6620796F757220637E
:102AB0006C6F636B2E0048657265206172652073D0
:102AC0006F6D65206F662074686520436C6F636B63
:102AD00020446973706C61797320737570706F72C4
:102AE00074656400416E616C6F6720436C6F636B4B
:102AF0002077697468206D696E696D616C20646906
:102B0000676974730000416E616C6F6720436C6F7E
:102B1000636B207769746820616C6C2064696769F5
:102B20007473000041646420746865203234206846
:102B30006F757273206E756D657269632064697359
:102B4000706C617900004F72206164642074686564
:102B500020414D2F504D206E756D65726963206464
:102B60006973706C617900004D697820616E642032
:102B70004D6174636820617320796F7520706C6596
:102B8000617365005475726E20746865204C45440D
:102B900020626C696E6B696E67206F666600416EBD
:102BA00064207475726E206974206261636B206F9B
:102BB0006E005475726E206F6E2043616C69627294
:102BC0006174696F6E204D6F646500005475726E9C
:102BD000206974206261636B206F66660000546830
:102BE0006520274127206F6E207468652073636F0E
:102BF0007065206D65616E732041565220436C6F85
:102C0000636B204D6173746572204D6F64650000C5
:102C10004D616B652054696D6520676F2066617337
:102C200074004D616B652054696D6520676F206E7F
:102C30006F726D616C004D616B652054696D65202C
:102C4000676F206261636B004D616B652054696D35
:102C50006520676F206261636B2066617374210079
:102C6000566572626F7365206F7574707574206934
:102C700073206F6E65206F6620796F7572206F709C
:102C800074696F6E730054686520626C696E6B695D
:102C90006E67204220776F756C6420696E6469638B
:102CA0006174652061206C6F77205254432062610B
:102CB000636B757020626174746572792C20627523
:102CC00074206E6F772069742773206A757374207F
:102CD000612064656D6F00005468697320626C69DF
:102CE0006E6B696E67205020696E646963617465FC
:102CF00073207468617420746865203120505053CB
:102D0000207369676E616C206973206D69737369E4
:102D10006E672E20416761696E2C206A757374207E
:102D2000612064656D6F000057696C6C2074686980
:102D3000732067657420796F757220617474656E95
:102D400074696F6E3F004275726E20696E207072FA
:102D50006576656E74696F6E206D6F76657320742D
:102D6000686520646973706C617920612074696E94
:102D700079206269742C206E6F726D616C6C7920A1
:102D800065766572792035206D696E75746573207E
:102D90006275742068657265206576657279207346
:102DA00065636F6E6400576520686F706520796F8A
:102DB0007520656E6A6F7965642074686973206434
:102DC000656D6F2E205468616E6B20796F7520667B
:102DD0006F72207573696E6720746869732044751B
:102DE00074636874726F6E697820436C6F636B00F4
:00000001FF
